:020000040000FA
:020000000528D1
:0800080067283420EB1F0E28CD
:10001000012282210624D126F22019289626031DCA
:1000200017280026031920288E24031920281C24B1
:10003000D722861EFC2AD81858214425031D2628BD
:100040004A25031D252882212628E92000250310A2
:10005000D20CD210851BD2145208013C031D192862
:100060001C24BD26F42019288B1394309F0083167E
:10007000031720308800890183160313831300308F
:100080009F009501C0308500E03086000030870079
:100090000030880007308900083081008312031384
:1000A0008313522412213325D401D301D801D20164
:1000B000D501D601C0010030F0005E25D000E2017C
:1000C000F601F701F801F7238B168B170800F200F1
:1000D000030EF3000408F4000A08F5000B11F60AF9
:1000E0007608FE3C031D7C28F601F70A7708103CD1
:1000F000031D7C28F7017814581D88280130D60785
:100100000318D50A5508023C031D8828D50118217B
:10011000122153086402031CB0284108E039C100D1
:1001200020305407840000081F39C10441088500AD
:100130004208E039C2002E305407840000081F39FD
:10014000C204420886005408C92087005408D920F8
:10015000C30443088800D40A54080E3C0319D40190
:10016000530A0339D300E20A62080A3C031DC0287F
:10017000E2015810891C5814D810091DD814D90A46
:1001800075088A0074088400730E8300F20E720EE4
:1001900009008A018207013402340434083410341F
:1001A00020344034803400340034003400340034CF
:1001B00000348A01820700340034003400340034F3
:1001C0000034003400340134023404340834103470
:1001D0002034500A0339D000F1000030F0006D25C2
:1001E000F22008005114F528511050088A018207A6
:1001F000FC28FE2800290929252308004C23080093
:100200000301511C8030C0002523C001511C742300
:1002100008000301511C8030C0004C23C001511C58
:10022000B923080087014308C039C30088000800CB
:10023000571C3F295710581E24293C08A0003D0890
:10024000A1003E08A2000800D81E2D293C08A400E9
:100250003D08A5003E08A6000800581F36293C08A6
:10026000AA003D08AB003E08AC000800D81F0800FB
:100270003C08AE003D08AF003E08B000080057142F
:10028000581E4629A001A101A2010800D81E4C2930
:10029000A401A501A6010800581F5229AA01AB011B
:1002A000AC010800D81F0800AE01AF01B001080082
:1002B0004808023C031C6321C801C901F220D81878
:1002C0005F2906240800C70A47080A3C031D0800E6
:1002D000C701C60A4608063C031D0800C601C50A38
:1002E0004508043C031D7B294408023C031D7B296F
:1002F000C501C401080045080A3C031D0800C501EA
:10030000C40A08005815C801C9012523D501D60122
:10031000D701C801C90158163C308400440808229E
:1003200058189029ED21D8189C29581C9229581842
:1003300097291A215812A529C40A03304402031927
:10034000C401ED21D818A2299229C41CAB29450863
:10035000033C031CC501D816F221D818B629581C35
:10036000A5295818B1291A21D812C129C50A043063
:10037000C41C0A3045020319C501F221D818BE2950
:10038000A5295817F721D818CC29581CC129581865
:10039000C7291A215813D529C60A0630460203195F
:1003A000C601F721D818D229C129D817FC21D8189D
:1003B000E029581CD5295818DB291A21D813E92916
:1003C000C70A0A3047020319C701FC21D818E629D9
:1003D000D52925230624581108003C308400440800
:1003E000082208003C3084004508082208003C3000
:1003F00084004608082208003C3084004708082290
:100400000800C401C501C601C701C801C90108002F
:10041000E300E1010430DA0013228000E10A840ADB
:10042000DA0B0C2A0800E108031D1A2A0310E30D59
:10043000630DE10002308A00610882071F34113425
:100440001F34003400341F34003400341D3415349C
:1004500017340034153415341F3400340734043491
:100460001F340034173415341D3400341F34153450
:100470001D34003401341D34033400341F3415346A
:100480001F340034173415341F3400341E3405343F
:100490001E3400341F3415340A3400340E34113441
:1004A000113400341F3411340E3400341F34153429
:1004B000153400341F34053405340034E300E00003
:1004C000E1010630DA006A228000E10A840ADA0BD0
:1004D000632A0800E108031D732A0310E30D630D6E
:1004E000E00D6007E10002308A00610882071F34D6
:1004F0001934193419341F3400341F340C340C34BB
:100500000C340E3400341F3401341F3418341F34BB
:1005100000341F3418341E3418341F340034183497
:1005200018341F341934193400341F3418341F346C
:1005300001341F3400341F3419341F3401341F3484
:1005400000340C340C34183418341F3400341F3485
:1005500019341F3419341F3400341F3418341F3435
:1005600019341F340034133413341F3413340E344D
:1005700000340F3413340F3413340F3400340E347A
:100580001334033413340E3400340F34133413345F
:1005900013340F3400341F3403341F3403341F3436
:1005A0000034033403340F3403341F3400348030F8
:1005B000C0005018DD2A2523DE2A4C23C0010F304D
:1005C000DE001C30DA00F1225A081F3E8400841736
:1005D0000008A0008413A6245A1CDE03DA0BE32AC9
:1005E00008001B30DB005B081F3E84000008840A03
:1005F0008000DB0BF32A0800D1262430DE001B30FC
:10060000DA005A08DB0021308400000884038000EF
:10061000840A840ADB0B052B84038001A624DE03F5
:10062000DA0B012B84031F308000152B0530DA0014
:100630001C30DB00203084000310800D840ADB0BAB
:100640001C2B8224DA0B182B080020304007840072
:10065000440803192D2B08222E2B3B234508082282
:10066000452346080822470808224523480808224F
:1006700049080822080003018000840A8000840AD7
:100680008000840A8000840A08000A308000840AFE
:1006900003018000840A08002030400784004708D6
:1006A0005E2246085E226A2345085E22440803193A
:1006B0005B2B5E2208005D2308008001840A800114
:1006C000840A8001840A8001840A8001840A8001EE
:1006D000840A08008001840A0A308000840A8001AC
:1006E000840A8001840A08000630DA0049084F02B3
:1006F000031D922348084E02031D962347084D020E
:10070000031D9A2346084C02031D9E2345084B02F5
:10071000031DA22344084A02031DA623A024DA0BCA
:10072000762B080038308400AA2308003430840077
:10073000AA2308002E308400AA2308002A3084004F
:10074000AA23080024308400AA2308002030840053
:10075000AA2308000330DB008417800CE001E00CC2
:10076000600C841380040310800C840ADB0BAC2B18
:1007700008000630DA0047084D02031DCF23460863
:100780004C02031DD32345084B02031DD723440805
:100790004A02031DDB23A024DA0BBB2B0800243004
:1007A0008400DF2308002A308400DF23080034306F
:1007B0008400DF2308003A308400DF2308000408A7
:1007C000E1000430DB00053061025A078400841721
:1007D0000008DF0084136108840084030008840A91
:1007E00080008403DB0BED2B5F08800008000F30D6
:1007F000E80049246908EB008E30E800E901442450
:100800008F30E800E9016916442408008030E800D0
:10081000480EE9004908E90444248130E800460E06
:10082000E9004708E90444248230E800440EE90066
:100830004508E904442408004408CA004508CB00E0
:100840004608CC004708CD004808CE004908CF0034
:100850000030E800492469080F39C900690E0F39D2
:10086000C8000130E800492469080F39C700690E43
:100870000F39C6000230E800492469080F39C50065
:10088000690E0F39C40008004E245E2461245224EE
:1008900008004E245E2470245224080043134308A9
:1008A000880008004317430888000800C313430862
:1008B00088000800C3174308880008006808EA0099
:1008C000632C6908EA000830DA005624C112EA1BDA
:1008D000C11641088500EA0D5A24DA0B652C080080
:1008E0000830DA00E90103105624E90D051B6914EC
:1008F0005A24DA0B742C08009830DC007F2CDC0BB7
:100900007E2C08002830DD007C24DD0B842C0800C0
:10091000F030DD007C24DD0B8A2C08002830E0005C
:1009200000254425031908008824E00B902C0311AE
:1009300008009830DC00861EFC2ADC0B9B2C08008B
:100940002830DD009924DD0BA22C08005E08DD00B4
:080950007C24DD0BA82C08003B
:100A00001F142E259F149F18032D1F101E0E0F3923
:100A1000E6006702031908000318132D013066026F
:100A2000031C0301142D6608E5001A25E40066087E
:100A3000E700080005308A006508820703340334A4
:100A400003340334033402340234023402340134F4
:100A50000134013400340034003400341430DA003E
:100A6000DA0B302D08001C30DA00203084008001C1
:100A7000840ADA0B372D1C30DA00A03084008001A4
:100A8000840ADA0B3F2D08000311581C08000315D7
:100A9000D90108000311581C08005125031D4A2DD7
:100AA00008005908FA3C0800002520308400660838
:100AB00008222430840064080822080083120317E7
:100AC00070088D00831603178C130C148312031700
:100AD0000C08831203138313080083120317700892
:100AE0008D0071088C00831603178C130C158B1363
:100AF0008B1B772D55308D00AA308D008C148B17F1
:100B0000000000000C118B178312031383130800DD
:100B10000130A0000230A1000430A2000830A30080
:100B20001030A4000830A5000430A6000230A70051
:100B30000130A8000230A9000430AA000830AB0040
:100B40001030AC000830AD001F30AE001E30AF00DA
:100B50001C30B0001830B1001030B2001830B300B3
:100B60001C30B4001E30B5001F30B6001E30B70078
:100B70001C30B8001830B9001030BA001830BB0073
:020B800008006B
:100C00007E26EE01EC01ED012E3084000025861ECB
:100C1000FC2A0019042E043080002326800184035E
:100C2000442503190800781C072E78100408E000FA
:100C3000292660088400EE0A6E08AD3C031D072ECD
:100C4000AF01031108000E30DD007C24DD0B252EE2
:100C50000800F601F701F801682630264926080049
:100C60006D0876266F08DF000310DF0D6C083B3C33
:100C700084003B26080006308A005F0882070011C6
:100C80000800801008008011080000100800001201
:100C900008006D0876266F08DF0020306C0784009E
:100CA00056268000840A5F268000080006308A00ED
:100CB0005F08820706340E340E340F341F340630BA
:100CC0008A005F088207003400340434043404349A
:100CD000EC01ED016E08DF000F30DF02031C722E05
:100CE000EC0A6C2E0F305F07ED000800DF00EF010B
:100CF0000330DF02031C0800EF0A782E0B30DA0005
:100D00003B3084001F3080008403DA0B822E0E30CB
:100D1000800084030430800084030F30DA008001F7
:100D20008403DA0B8F2E0430A0000800E926062782
:100D30007908FC007A08FD007B08FE001C240627C9
:100D4000AE26FB1BAA2E0330FC00FD01FE01AE26E1
:100D5000FB1BAC2E03110800031508007C08F902E8
:100D60000130031CFA02031CFB027D08FA02013069
:100D7000031CFB027E08FB020800C408031D0800D8
:100D8000C508031D0800C608031D0800C708031D89
:100D90000800C808031D0800C908031D0800D12663
:100DA000080028249830E8004424E90144249930BC
:100DB000E800480EE9004908E9044424460EE90029
:100DC0004708E9044424440EE9004508E9044424A2
:100DD00008009830E8004424E90144241930E80070
:100DE000492469080F39C900690E0F39C800492420
:100DF00069080F39C700690E0F39C6004924690810
:100E00000F39C500690E0F39C4000800F901FA0155
:100E1000FB014908F9004808DF004027F9070310E3
:100E2000470DDF004A27F9070318FA0ADF0A4A27A5
:100E3000FA070310460DDF006227F9070318FA0AC4
:100E4000DF0A6227FA070310450DDF007227F90752
:100E50000318FA0ADF0A7227FA074408DF000310B2
:100E6000DF0D0310DF0D8A27F9070318FA0ADF0ADE
:100E70008A27FA070318FB0ADF0A8A27FB070800FC
:100E800007308A005F08820700340A3414341E34A5
:100E90002834323407308A005F0882070034003477
:100EA0003C34003478340034B4340034F03400344A
:100EB0002C34013468340134A4340134E034013476
:100EC0001C34023407308A005F0882070034003483
:100ED0003A340234B034043408340734603409340A
:100EE000B8340B3407308A005F08820700340034BE
:100EF00010340E3420341C3430342A344034383426
:100F00005034463460345434703462348034703435
:100F100090347E3407308A005F0882070034003442
:100F200000340034A0348C3400340034403419349C
:040F30000134003454
:02400E00C42FBD
:024010000000AE
:024200000000BC
:00000001FF
